:100000000C94A1030C94DB030C94DB030C94DB0332
:100010000C94DB030C94DB030C94DB030C94DB03E8
:100020000C94DB030C94DB030C94DB030C94DB03D8
:100030000C94DB030C94DB030C94DB030C94DB03C8
:100040000C94DB030C94DB030C94DB030C94DB03B8
:100050000C94DB030C94DB030C94DB030C94DB03A8
:100060000C94DB030C94640D0C94DB030C94930D43
:100070000C94DB030C94D7220C94DB030C94DB036D
:100080000C94DB030C94DB030C94DB030C94DB0378
:100090000C94DB030C94DB030C94DB030C94DB0368
:1000A0000C94DB030C94DB030C94DB030C94DB0358
:1000B0000C94DB030C94DB030C94DB030C94330CE7
:1000C0000C94DB030C94DB030C94DB030C94DB0338
:1000D0000C94DB030C94DB030C94DB030C94DB0328
:1000E0000C94DB030C94D0060C94E5060C942D06BE
:1000F0000C9461060C9420070C94DB030C94BE0650
:100100000C94DB030C94DB030C94DB030C94DB03F7
:100110000C94DB030C94DB030C94DB030C94F706C8
:1001200045464765666700202B2D2E30313233342B
:10013000353637383968000A7472616E736D6973C9
:1001400073696F6E206661696C65642C206D7573D0
:100150007420626520696E20504C4C5F4F4E2073B6
:10016000746174650A000A7472616E736D6974203B
:100170006572726F723A206461746120657863659C
:100180006564656420313235206279746573002EB0
:100190000A2053656520576562626F744C6962205E
:1001A0006D616E75616C206F6E2066696C654F7055
:1001B000656E20696E2046696C6553797374656D50
:1001C0002F4641542E6820666F72206D6F72652035
:1001D000696E666F2E0A00546865206D6F64652035
:1001E000706172616D6574657220697320696E76E5
:1001F000616C69640020342E204953502050726F86
:100200006772616D6D657220697320706C756767C8
:10021000656420696E0020332E205468652066696D
:100220006C6520616C7265616479206578697374AE
:10023000732062757420617320616E20696E636F34
:100240006D70617469626C6520656E636F64696E60
:10025000670A0020322E20546865207553442063BD
:10026000617264206973206E6F7420696E207468F7
:100270006520736C6F740A0020312E20546865204D
:100280006469736B2069732066756C6C0A00457233
:10029000726F722063617573656420627920616E8C
:1002A0007920636F6D62696E6174696F6E206F662D
:1002B0002074686573653A0A00596F75206172652C
:1002C00020747279696E6720746F20777269746523
:1002D00020746F20612072656164206F6E6C7920DC
:1002E00066696C6500546865206469726563746F43
:1002F000727920646F65736E2774206578697374F2
:10030000005468652066696C6520616C7265616483
:100310007920657869737473207768656E206F70D3
:10032000656E696E6720666F72207772697465000A
:100330005468652066696C6520646F65736E277408
:10034000206578697374207768656E206F70656EBC
:10035000696E6720666F722072656164000A436F80
:10036000756C646E277420637265617465206669BC
:100370006C652C206572726F723A2025640A200029
:100380000A525353493A25642045443A2564205281
:100390004E443A25640A002563000A676F696E6758
:1003A00020696E746F205258206D6F64650A000AD0
:1003B000656E746572696E67207472616E736D69C3
:1003C00074206D6F64650A00616463315F53686116
:1003D00072703A2025642C2074696D6520286D7335
:1003E000293A2025640A000A45443A25640A000A8D
:1003F000524553455454494E47000A2564000A6744
:100400006F696E6720696E746F205258206D6F643B
:1004100065000A726573657420636F6D6D616E644B
:100420002073656E7420776972656C6573736C797F
:10043000000A656E746572696E67207472616E730E
:100440006D6974206D6F64650A70757368206275DC
:1004500074746F6E20746F2072657365742072659A
:100460006D6F746520756E69740A000A0A41786FB1
:100470006E204D6F746520696E697469617465647E
:100480002E0A5472616E736D6974206F6E2043681A
:10049000616E6E656C2025642E0A0A00F502006EFE
:1004A00000024700350002440006AE06F902006E65
:1004B000000448003500044400040000FD02016F00
:1004C00000028800360002800006A8060103016FC2
:1004D00000048A00360004800004AB060503016FA7
:1004E00000088C00360008800002AE060903027086
:1004F0000002B300370002B0000600000D030270D6
:100500000004B400370004B00004000011030371BC
:1005100000029800380002900006C006150303711F
:1005200000049A00380004900004C3061903037104
:1005300000089C00380008900002C6061D030472E3
:100540000002A800390002A0000600002103047286
:100550000004AA00390004A000040000250304726E
:100560000008AC00390008A0000200002903057350
:10057000000228013A000220010600002D03057345
:1005800000042A013A00042001040000310305732D
:1005900000082C013A000820010200003503460043
:1005A0004500000002338844000144000245000871
:1005B0000000019C046E00013500010000000001F4
:1005C0000000010000010000400384008100FF00E2
:1005D00003FFDF800001800002810008810010BC61
:1005E000046F000136000186006F00203600208174
:1005F000004000004B03B200B1000000023388B09D
:100600000001B00002B10008000001EC047000011C
:10061000370001000000000100000100000100009F
:10062000560394009100FF0003FFDF90000190004B
:10063000029100089100100C05710001380001962C
:1006400000710020380020910040CC066103A40016
:10065000A100FF0003FFDFA00001A00002A100082D
:10066000A100103C05720001390001A600720020B3
:10067000390020A1004000006C0324012101FF008B
:1006800003FFDF2001012001022101082101106C7C
:10069000057300013A000126017300203A00202171
:1006A0000140000051026D02D70620D70640D70650
:1006B00080DD0608DD0680E30601E30602E30604AA
:1006C000E30608E30610E30620E30640E30680E9BC
:1006D0000601EF0602E40C2500240023002B002A6B
:1006E0000029002E002D002C00310030002F003496
:1006F0000033003200470E3F0E1B217F20131F5591
:10070000736572204572726F723A25640A005765EC
:1007100062626F744C6962204572726F723A25642E
:100720000A002228C427F127C827D127592800000A
:10073000000000006F29252A412AFA292C2A102AB4
:10074000E62211241FBECFEFD1E4DEBFCDBFE4E52A
:10075000F0E080818093ED04E4E5F0E0108288E130
:100760000FB6F89480936000109260000FBE12E004
:10077000A0E0B2E0E2E6F0E600E00BBF02C00790C6
:100780000D92A83EB107D9F714E0A8EEB2E001C07F
:100790001D92AD3EB107E1F717E0C2E4D7E004C017
:1007A0002297FE010E942B30C034D107C9F70E9466
:1007B00022250C94DE2E0C940000DF93CF93CDB74E
:1007C000DEB7EDE4F1E08081877F8083EEE4F1E045
:1007D000808181608083EEE4F1E0808182608083AB
:1007E000EEE4F1E0808184608083EEE4F1E08081DA
:1007F00088608083EEE4F1E0808180648083EEE4B1
:10080000F1E0808180618083E1E5F1E080818F7B90
:100810008083E1E5F1E0808180618083E1E5F1E0C2
:10082000809100028F70982F9F708081807F892B2C
:100830008083E4E4F1E0808180628083E5E4F1E09C
:100840008081807F8083E5E4F1E080818063808324
:10085000E5E4F1E08081806C8083ECE4F1E080816C
:100860008C7F8083CF91DF910895DF93CF93CDB7B5
:10087000DEB7E1E4F1E080818F718F31D1F3CF9168
:10088000DF910895DF93CF93CDB7DEB70E94350493
:10089000A9E3B1E0E9E3F1E080818D7F8C930E94D0
:1008A0003504A9E3B1E0E9E3F1E0808181608C9354
:1008B000E1E4F1E080818F718830D1F70E94DD039F
:1008C0007894CF91DF910895DF93CF93CDB7DEB7C2
:1008D000E2E4F1E08081807E88608083CF91DF91C7
:1008E0000895DF93CF930F92CDB7DEB789830E942F
:1008F00035048981813081F4E1E4F1E080818F71F8
:10090000883021F00E9464040E943504E9E3F1E09C
:1009100080818260808308C08981882329F4E9E38B
:10092000F1E080818D7F80830F90CF91DF910895DA
:10093000DF93CF930F92CDB7DEB7898389818B3058
:1009400018F48BE0898305C089818B3110F08AE12E
:100950008983E8E4F1E089818F71982F9F7180810C
:10096000807E892B808369E170E080E090E00E94C6
:1009700002290F90CF91DF910895DF93CF930F92CB
:10098000CDB7DEB71982A8E4B1E0E8E4F1E08081F8
:1009900080688C936CE870E080E090E00E9402290F
:1009A000E8E4F1E080818F71898389810F90CF9194
:1009B000DF910895DF93CF93CDB7DEB70E94350462
:1009C000E2E4F1E08081807E896080836EE670E001
:1009D00080E090E00E940229EFE4F1E080818170E4
:1009E0008823D1F7CF91DF910895DF93CF93CDB7CF
:1009F000DEB70E943504E1E4F1E080818F71883038
:100A000069F41092EF02E2E4F1E08081807E86607A
:100A100080838091EF028823E1F30CC0E1E4F1E0F0
:100A200080818F71893031F4E2E4F1E08081807E51
:100A300086608083E1E4F1E080818F718630D1F7B8
:100A4000CF91DF910895DF93CF93CDB7DEB70E94AA
:100A500035048FEF8093EE02E1E4F1E080818F7145
:100A6000893069F4E2E4F1E08081807E82608083F5
:100A70008091EE028823E1F71092EB0210C087E329
:100A800091E000D00F92EDB7FEB7319621E02083C0
:100A9000928381830E94B2250F900F900F900E9445
:100AA0003504E2E4F1E08081807E89608083CF912B
:100AB000DF910895DF93CF930F92CDB7DEB789838F
:100AC0008091EB028F5F8093EB02E0E8F1E0809190
:100AD000EB028E5F80838091EB02882F90E080583C
:100AE0009E4FFC01898180830F90CF91DF91089503
:100AF000DF93CF9300D0CDB7DEB79A838983898106
:100B00009A81009799F12DC08091EB028F5F8093BD
:100B1000EB028091EB028E3780F48091EB02882FFC
:100B200090E080589E4FDC01E981FA8180818C93AE
:100B300089819A8101969A8389838091EB028E370D
:100B400081F486E691E000D00F92EDB7FEB73196C2
:100B500021E02083928381830E94B2250F900F9021
:100B60000F90E981FA818081882371F6E0E8F1E055
:100B70008091EB028E5F80830F900F90CF91DF9179
:100B80000895DF93CF93CDB7DEB7E6E4F1E080813F
:100B90008F718093E802E6E4F1E08081829586958A
:100BA0008770837080932404CF91DF910895DF9341
:100BB000CF93CDB7DEB70E94DA04CF91DF910895CD
:100BC000DF93CF93CDB7DEB70E942305CF91DF919E
:100BD0000895DF93CF93CDB7DEB70E94F504CF9190
:100BE000DF910895DF93CF930F92CDB7DEB789835E
:100BF0008981813019F40E94DA0402C00E94F50450
:100C00000F90CF91DF910895DF93CF93CDB7DEB7EB
:100C10000E946404CF91DF910895DF93CF93CDB705
:100C2000DEB781E00E947104CF91DF910895DF93D8
:100C3000CF93CDB7DEB780E00E947104CF91DF91F2
:100C40000895DF93CF93CDB7DEB7E0E8F1E01082EF
:100C50001092EB02CF91DF9108951F920F920FB681
:100C60000F9200905B000F9211242F933F934F93AC
:100C70005F936F937F938F939F93AF93BF93EF9304
:100C8000FF93DF93CF93CDB7DEB70E94C105E7E4B2
:100C9000F1E08FEF8083CF91DF91FF91EF91BF91D2
:100CA000AF919F918F917F916F915F914F913F9104
:100CB0002F910F9000925B000F900FBE0F901F902E
:100CC00018951F920F920FB60F9200905B000F9233
:100CD00011242F933F938F939F93EF93FF93DF9371
:100CE000CF9300D0CDB7DEB7E6E4F1E08081807825
:100CF000882381F11A821982EBE7F1E080818A83EF
:100D0000198211C08981282F30E08981882F90E0D5
:100D100080589E4FFC018081F901EB5DFB4F808381
:100D200089818F5F89838981282F30E08A81882F8C
:100D300090E00297281739072CF38A81882F90E0DA
:100D400080589E4FFC0180818093EA028FEF809350
:100D5000EC0202C01092EC020F900F90CF91DF9145
:100D6000FF91EF919F918F913F912F910F90009262
:100D70005B000F900FBE0F901F9018951F920F925F
:100D80000FB60F921124DF93CF93CDB7DEB7109239
:100D9000EE02CF91DF910F900FBE0F901F9018952C
:100DA0001F920F920FB60F9211248F93DF93CF9360
:100DB000CDB7DEB78FEF8093EF02CF91DF918F91A8
:100DC0000F900FBE0F901F9018951F920F920FB6A5
:100DD0000F921124DF93CF93CDB7DEB71092EF02BD
:100DE000CF91DF910F900FBE0F901F9018951F921B
:100DF0000F920FB60F9200905B000F9211248F9309
:100E0000EF93FF93DF93CF93CDB7DEB7E1E5F1E04A
:100E100080818F7B80838FEF8093ED02E1E5F1E0AD
:100E2000808180648083CF91DF91FF91EF918F91DA
:100E30000F9000925B000F900FBE0F901F901895BF
:100E40001F920F920FB60F9200905B000F92112429
:100E50008F93EF93FF93DF93CF93CDB7DEB7E7E4A4
:100E6000F1E080818093E902CF91DF91FF91EF91D2
:100E70008F910F9000925B000F900FBE0F901F900C
:100E80001895DF93CF930F92CDB7DEB789834DE5E9
:100E900053E08981282F332727FD309500D000D0DB
:100EA0000F92EDB7FEB7319681E080835283418384
:100EB000348323830E94B2250F900F900F900F90E0
:100EC0000F9089818F3F81F480E393E000D00F92EF
:100ED000EDB7FEB7319621E02083928381830E9493
:100EE000B2250F900F900F9089818E3F81F481E0A1
:100EF00093E000D00F92EDB7FEB7319621E020834A
:100F0000928381830E94B2250F900F900F90898168
:100F10008D3F81F485EE92E000D00F92EDB7FEB7E1
:100F2000319621E02083928381830E94B2250F9025
:100F30000F900F9089818C3F81F489EB92E000D073
:100F40000F92EDB7FEB7319621E020839283818323
:100F50000E94B2250F900F900F9089818B3F09F06E
:100F600050C02EE832E000D00F92EDB7FEB73196B8
:100F700081E08083328321830E94B2250F900F90FD
:100F80000F9028E732E000D00F92EDB7FEB7319610
:100F900081E08083328321830E94B2250F900F90DD
:100FA0000F9023E532E000D00F92EDB7FEB73196F7
:100FB00081E08083328321830E94B2250F900F90BD
:100FC0000F9026E132E000D00F92EDB7FEB73196D8
:100FD00081E08083328321830E94B2250F900F909D
:100FE0000F9025EF31E000D00F92EDB7FEB73196AC
:100FF00081E08083328321830E94B2250F900F907D
:101000000F9089818A3F81F487ED91E000D00F92A3
:10101000EDB7FEB7319621E02083928381830E9451
:10102000B2250F900F900F90898188232CF48AE4C9
:1010300092E00E94340804C08AE492E00E944508CD
:101040008FE891E000D00F92EDB7FEB7319621E026
:101050002083928381830E94B2250F900F900F907E
:101060000F90CF91DF910895DF93CF9300D0CDB74C
:10107000DEB79A83898389819A816FEF0E94002568
:101080000F900F90CF91DF910895DF93CF9300D011
:10109000CDB7DEB79A83898389819A8160E00E9407
:1010A00000250F900F90CF91DF910895DF93CF939C
:1010B0000F92CDB7DEB7809123048130F9F48FEA27
:1010C00093E000D00F92EDB7FEB7319621E0208378
:1010D000928381830E94B2250F900F900F900E94FF
:1010E000D70568EE73E080E090E00E94270982E077
:1010F00092E00E9478050E94E005F3CF80912304DE
:10110000882309F0A0C08AE993E000D00F92EDB7E0
:10111000FEB7319621E02083928381830E94B2251D
:101120000F900F900F900E94E90560ED77E080E04E
:1011300090E00E9427098091EC028823B1F181E0C0
:101140000E94F205198221C047E953E08981882F66
:1011500090E0FC01EB5DFB4F8081282F30E000D058
:1011600000D00F92EDB7FEB7319681E080835283B5
:101170004183348323830E94B2250F900F900F90F8
:101180000F900F9089818F5F89838981282F30E0AC
:1011900080912604882F90E0029728173907A4F23F
:1011A0000E94210680E00E94F205A0E8B3E0809151
:1011B000E802282F30E08091E902482F50E080912A
:1011C0002404682F70E08DB79EB709970FB6F89486
:1011D0009EBF0FBE8DBFEDB7FEB7319681E0808315
:1011E000B283A183348323835683458370876783C7
:1011F0000E94B2258DB79EB709960FB6F8949EBF90
:101200000FBE8DBF8091E902882329F080EE94E023
:101210000E94340804C080EE94E00E94450880914A
:10122000EC02882329F08AE492E00E94340804C08A
:101230008AE492E00E9445081092EC021092E902C2
:101240001092E80272CF0F90CF91DF910895DF9353
:10125000CF9300D000D0CDB7DEB769837A838B837C
:101260009C8389819A81AB81BC81BC01CD010E94A4
:10127000B9230F900F900F900F90CF91DF910895A9
:10128000EF92FF920F931F93DF93CF93CDB7DEB70B
:101290002A970FB6F894DEBF0FBECDBF0E940F0C89
:1012A000DC01CB018F839887A987BA878BE692E010
:1012B0000E94D709882309F45FC0809123048130FC
:1012C00009F05AC080EE94E00E94340881E00E9448
:1012D000A7229E838D830E940F0C9B01AC018F81FE
:1012E0009885A985BA8579018A01E81AF90A0A0B55
:1012F0001B0BD801C70128EE33E040E050E0BC01F1
:10130000CD010E94EC2FDA01C90189839A83AB8356
:10131000BC8328EC33E00DB71EB7095010400FB660
:10132000F8941EBF0FBE0DBFEDB7FEB7319681E03A
:101330008083328321838D819E81948383838981FD
:101340009A81AB81BC8185839683A783B0870E94F5
:10135000B2258DB79EB709960FB6F8949EBF0FBE03
:101360008DBF68EC70E080E090E00E94270980EE7D
:1013700094E00E9445089ACF8BE692E00E94D7093C
:10138000882309F493CF80912304882309F08ECF1A
:101390008AE492E00E94340868EC70E080E090E01B
:1013A0000E9427098AE492E00E9445087FCFDF93DC
:1013B000CF9300D00F92CDB7DEB79A838983E981AE
:1013C000FA81808191810E9488241B82882311F4F4
:1013D00081E08B838B810F900F900F90CF91DF91E5
:1013E0000895DF93CF93CDB7DEB78DE692E061E845
:1013F0000E94332368EE73E080E090E00E942709AA
:101400008DE692E06FE70E94332368EE73E080E0A0
:1014100090E00E942709CF91DF910895DF93CF9349
:101420000F92CDB7DEB788E192E00E94772A8983D8
:1014300089818F3F41F18981813349F48DE692E0C2
:1014400061E80E9433238AE492E00E943408898193
:10145000823349F48DE692E06FE70E94332380EEF9
:1014600094E00E9434088981833369F48DE692E028
:1014700060E00E9433238AE492E00E94450880EEF7
:1014800094E00E9445080F90CF91DF910895DF937B
:10149000CF93CDB7DEB7809123048130E1F580EEA4
:1014A00094E00E9434088AE492E00E94450821E317
:1014B00034E000D00F92EDB7FEB7319681E0808323
:1014C000328321830E94B2250F900F900F900E94CB
:1014D000D70566E970E080E090E00E9427098BE67E
:1014E00092E00E94D7098823A1F382E00E945A0566
:1014F00082E194E000D00F92EDB7FEB7319621E083
:101500002083928381830E94B2250F900F900F90C9
:101510000E94E005DECF80912304882309F07CC07F
:101520008AE492E00E94340880EE94E00E9445082C
:101530002EEF33E000D00F92EDB7FEB7319681E089
:101540008083328321830E94B2250F900F900F90E9
:101550000E94E90581E00E94F2054AEF53E0809184
:101560002504282F30E000D000D00F92EDB7FEB751
:10157000319681E0808352834183348323830E94A8
:10158000B2250F900F900F900F900F90809125042F
:101590008230D9F42FEE33E000D00F92EDB7FEB7D2
:1015A000319681E08083328321830E94B2250F909F
:1015B0000F900F9088E190E02CE00FB6F894A8957A
:1015C000809360000FBE209360000E94210680E09F
:1015D0000E94F2051092250447EE53E08091E90243
:1015E000282F30E000D000D00F92EDB7FEB7319633
:1015F00081E0808352834183348323830E94B22518
:101600000F900F900F900F900F9060ED77E080E0BB
:1016100090E00E9427099ECFCF91DF910895DF933C
:10162000CF93CDB7DEB78BE692E00E94D70988232F
:1016300091F080912304882371F48AE492E00E945F
:10164000340868EC70E080E090E00E9427098AE4AA
:1016500092E00E944508CF91DF910895DF93CF93E8
:10166000CDB7DEB70E94FD0CCF91DF9108950F93A7
:101670001F93DF93CF9300D000D0CDB7DEB769833F
:101680007A838B839C8364E670E080E090E00E9424
:1016900027098FE492E00E94D709882339F080EE71
:1016A00094E00E94340881E0809323048DE492E06A
:1016B0000E94D709882331F08AE492E00E9434081E
:1016C0001092230464E670E080E090E00E94270915
:1016D0000E944204809101020E9498040BE614E0EB
:1016E0000E94BD04282F30E000D000D00F92EDB74B
:1016F000FEB7319681E08083128301833483238394
:101700000E94B2250F900F900F900F900F9080E0E5
:1017100090E0A0E0B0E0BC01CD010F900F900F90E1
:101720000F90CF91DF911F910F910895DF93CF9389
:10173000CDB7DEB728970FB6F894DEBF0FBECDBF8A
:1017400069837A838B839C832D833E834F83588761
:101750000E94400980E090E0A0E0B0E0BC01CD0133
:1017600028960FB6F894DEBF0FBECDBFCF91DF91A4
:101770000895FC016FB7F8948091240190912501A0
:101780002091F0023091F1024091F2025091F30267
:10179000208331834283538320912401309125019A
:1017A000358324832817390710F0D19B12C080811C
:1017B0009181A281B38180509348AF4FBF4F808306
:1017C0009183A283B3838091240190912501958315
:1017D00084836FBF0895EF92FF920F931F93FC01D4
:1017E000E080F180028113816481758180E090E066
:1017F00020E03DE740E050E00E94B92F20E03AEFC2
:1018000040E050E00E94EC2F2E0D3F1D401F511F65
:10181000B901CA011F910F91FF90EF9008950F93A6
:101820001F93DF93CF9300D000D000D0CDB7DEB7A9
:101830008E010F5F1F4FC8010E94B90BC8010E94A3
:10184000EB0B26960FB6F894DEBF0FBECDBFCF913F
:10185000DF911F910F910895D19AE3E7F0E0808125
:101860008260808308951F920F920FB60F92112409
:101870002F938F939F93AF93BF938091F00290919A
:10188000F102A091F202B091F30280509348AF4F61
:10189000BF4F8093F0029093F102A093F202B093B5
:1018A000F3022091DB042223B9F1579B35C08091CC
:1018B000F402882319F081508093F4028091F4029D
:1018C000882351F58091DC04882359F4822F9927CD
:1018D00087FD909597FF03C0909581959F4F8093CA
:1018E000DC0427FD02C09FE001C097E02091DD04E9
:1018F000222341F08091DC0481508093DC04882312
:1019000009F49EE31092DD04222319F481E0809310
:10191000DD049093F4024F9ABF91AF919F918F9104
:101920002F910F900FBE0F901F901895E8ECF5E0E7
:10193000A591B4918EE01A968C931A97E0E8F0E0A6
:10194000808182608083E1E8F0E08081886080832C
:1019500080818061808380E49CE9909387008093FC
:10196000860028E030E02D933C9380818260808364
:10197000E8E7F6E0A591B49184E01A968C931A9763
:10198000E1E2F1E080818860808380E09AEF9093CB
:101990002901809328012D933C938081826080836C
:1019A0000895FB010484F585E02D309719F42FEF9D
:1019B0003FEF02C009959C01C9010895DC011C9606
:1019C000ED91FC911D97309719F42FEF3FEF02C076
:1019D00009959C01C901089584EB96E09093E10478
:1019E0008093E0048091E2048C7F8093E20480EE97
:1019F00094E06FEF0E940025089583E892E00E9432
:101A0000C90D81EB96E06FEF0E94D92408950F93E2
:101A10001F9380914D0290914E026FEF0E94B2246D
:101A200080914F02909150026FEF0E94B2248FE597
:101A300092E06FEF0E94172601E512E0C8010E94B4
:101A400021210E94191FAC0184EA94E061E0980111
:101A50000E94451D02EC1DE0C8010E942A248FE867
:101A600092E09093EC048093EB0410939C0200931B
:101A70009B02C8010E948C258DE992E09093EA04B4
:101A80008093E9041093AA020093A9028BEA92E0E2
:101A90009093E8048093E7048DEB9DE09093B80267
:101AA0008093B70288E192E040E054E863E070E0A0
:101AB0000E94292980916B0290916C026FEF0E9425
:101AC000B2241F910F9108951F920F920FB60F929B
:101AD0000BB60F9211242F933F934F935F936F9305
:101AE0007F938F939F93AF93BF93EF93FF93E09177
:101AF0004402F0914502608188E192E00E945D2AF3
:101B0000FF91EF91BF91AF919F918F917F916F91D5
:101B10005F914F913F912F910F900BBE0F900FBE91
:101B20000F901F9018951F920F920FB60F920BB641
:101B30000F9211242F933F934F935F936F937F9353
:101B40008F939F93AF93BF93EF93FF9388E192E0BE
:101B50000E94162BFF91EF91BF91AF919F918F91B2
:101B60007F916F915F914F913F912F910F900BBE9D
:101B70000F900FBE0F901F90189588E192E00E9481
:101B8000772A0895682F88E192E00E940C2B90E05C
:101B900008958F929F92AF92BF92CF92DF92EF9271
:101BA000FF920F931F93CF93DF936C01DC0112968A
:101BB0008C91C82FD0E021977E01EE0CFF1C95EF91
:101BC000892E96E0992E8CE2A82E47C0D601ED9181
:101BD000FC91EE0DFF1D05911491F801D582C48290
:101BE000868197810E945F28FC01D80155969C93BD
:101BF0008E9354973296B49011969C928E9216962C
:101C00008D919C91179760E00E94D924BA9CC001E5
:101C1000112485549A4FFC01A591B4918D919C910A
:101C2000D80153969C938E93529718966D917C9100
:101C300019971A964D915C911B97C8010E94650EE9
:101C4000C80160E00E943323C8016FEF0E94532354
:101C50002197EEEFFFEFEE0EFF1EFFEFCF3FDF0706
:101C600009F0B4CFDF91CF911F910F91FF90EF90CA
:101C7000DF90CF90BF90AF909F908F900895FC0120
:101C800084899589611162E00E94AB280895EF92E2
:101C9000FF920F931F93FC01E488F5882485358516
:101CA00006851785862F992787FD909561E87FEF38
:101CB0004FE750E00E94E623BC01C7010E94CD28F7
:101CC0001F910F91FF90EF9008959F92AF92BF9256
:101CD000CF92DF92EF92FF920F931F93CF93DF93F8
:101CE000EC017B018A01798768875B874A878C8151
:101CF0009D81892B09F45EC09FB6F8948A899B89DF
:101D000068EE73E00E94D82F5B01CC24DD24B7017C
:101D1000601B710B80E090E0A60195010E94B92F35
:101D200024E130E040E050E00E94EC2FC901DA01EC
:101D30009C01AD01DA01C901807090700097A10586
:101D4000B10539F086EE0E942F242FEF3FEF40E0DF
:101D500050E03D872C870E0D1F1DB80180E090E0FC
:101D6000A60195010E94B92F24E130E040E050E047
:101D70000E94EC2FC901DA019C01AD01DA01C90111
:101D8000807090700097A105B10539F086EE0E9431
:101D90002F242FEF3FEF40E050E03F872E878B81CD
:101DA00080FF07C06A8161506A836F5FCE010E9425
:101DB00033239FBEDF91CF911F910F91FF90EF9042
:101DC000DF90CF90BF90AF909F900895AF92BF9259
:101DD000CF92DF92EF92FF920F931F93CF93DF93F7
:101DE000EC015A016B016B8970E080E090E02A8D74
:101DF0003B8D4C8D5D8D0E94B92F7B018C018989B3
:101E00009A89A0E0B0E0E80EF91E0A1F1B1F8EA100
:101E1000803269F08C899D8924E0969587952A9572
:101E2000E1F7A0E0B0E0E80EF91E0A1F1B1F8EEFDD
:101E30009FEFAFEFBFEFA80EB91ECA1EDB1E2889A9
:101E400030E040E050E0C601B5010E94B92F9B018F
:101E5000AC012E0D3F1D401F511FB901CA01DF917A
:101E6000CF911F910F91FF90EF90DF90CF90BF9097
:101E7000AF900895EF92FF920F931F93CF93DF934C
:101E80008C01EB01898190E0DC01AA0FBB1FA80F38
:101E9000B91F1196AA0FBB1FAC0FBD1F15968C91D1
:101EA000159781FF34C0F801808191810296FC0171
:101EB000E590F4904D915D916D917C919E01265E2F
:101EC0003F4FF80182819381F70109958823F9F04A
:101ED0008981282F30E0C9010196FC01EE0FFF1F18
:101EE000E80FF91FEE0FFF1FEC0FFD1F8081882305
:101EF00061F4F901EE0FFF1FE20FF31FEE0FFF1F5A
:101F0000EC0FFD1F87818D7F87838FEF01C080E0FD
:101F1000DF91CF911F910F91FF90EF9008956F92F5
:101F20007F928F929F92AF92BF92CF92DF92EF9269
:101F3000FF920F931F93CF93DF934C01FC01A68078
:101F4000B780C084D184E68CF78C00A111A1EA0C83
:101F5000FB1C0C1D1D1DEA14FB040C051D0538F4AB
:101F6000C701B80186017501DB015C016D01F40157
:101F7000C4A9D5A966246A94772425C0898190E0F4
:101F8000FC01EE0FFF1FE80FF91F3196EE0FFF1F48
:101F9000EC0FFD1F80819181A281B3818A159B0581
:101FA000AC05BD0568F0E816F9060A071B0740F006
:101FB000858181FF05C0C401BE010E943A0F6822DD
:101FC0007394C65EDD4FF40183A97816B8F2862DAE
:101FD000DF91CF911F910F91FF90EF90DF90CF9005
:101FE000BF90AF909F908F907F906F900895CF9209
:101FF000DF92EF92FF920F931F93CF93DF936C01C9
:10200000EB0179018A01FC0180819181FC01A5919C
:10201000B4919B01265E3F4FF60182819381B80106
:10202000A701FD0109958823F9F0898190E0FC0161
:10203000EE0FFF1FE80FF91FEE0FFF1FEC0FFD1F44
:10204000878181608783898190E0FC01EE0FFF1F0B
:10205000E80FF91F3196EE0FFF1FEC0FFD1FE08216
:10206000F182028313838FEFDF91CF911F910F9144
:10207000FF90EF90DF90CF9008950F931F93CF9331
:10208000DF938C01FC01C4A9D5A933A920E008C0C5
:10209000CE014A966817790739F02F5FC65EDD4F8B
:1020A0002317B0F3C0E0D0E0898190E00196FC01F5
:1020B000EE0FFF1FE80FF91FEE0FFF1FEC0FFD1FC4
:1020C0008081882311F0815080834981242F30E062
:1020D000C9010196FC01EE0FFF1FE80FF91FEE0F7B
:1020E000FF1FEC0FFD1F8081882361F5442351F110
:1020F000F901EE0FFF1FE20FF31F3196EE0FFF1FE6
:10210000EC0FFD1F858181FF04C0C801BE010E9444
:102110003A0F89818150843008F48983898190E065
:10212000FC01EE0FFF1FE80FF91F3196EE0FFF1FA6
:10213000EC0FFD1F2081318142815381C801BE0116
:102140000E94F70FDF91CF911F910F910895EF92A9
:10215000FF920F931F93FC0186A18031B1F0803272
:10216000C9F08C3099F57A018B01EE0CFF1C001F31
:10217000111FE40EF51E061F171F8AE0169507951E
:10218000F794E7948A95D1F70EC0E52EF62E072F27
:10219000112709C07A018B01A7E016950795F794DE
:1021A000E794AA95D1F7828D938DA48DB58DE8160D
:1021B000F9060A071B0750F4818992899C0140E0C7
:1021C00050E02E0D3F1D401F511F04C020E030E0A5
:1021D00040E050E0B901CA011F910F91FF90EF90CC
:1021E0000895FC0186A1803129F0803269F08C309D
:1021F00081F405C02FEF3FEF40E050E00EC02FEF1D
:102200003FE040E050E009C02FEF3FEF4FEF5FE0CD
:1022100004C020E030E040E050E0B901CA01089578
:10222000982F81568A3110F490520EC09D3261F081
:102230009F3551F09E3741F0892F80538A3020F02E
:1022400081518A3108F09FE5892F0895FC01CB0167
:10225000AA27BB27958B848B538F428F0895FC014F
:1022600088E1DF011D928A95E9F7408751876287EF
:10227000738744875587668777870895DF92EF9243
:10228000FF920F931F93CF93DF93EC017B01CB0160
:1022900060E270E04BE050E00E94F92E88818E32BF
:1022A00021F000E0DD2410E02BC0F7018083CE0197
:1022B000019629812E32E1F52183CE01029638C0A4
:1022C0008E3229F4002329F40FEF18E018C0002300
:1022D00059F01B3038F40E941011F701E10FF11D85
:1022E00080831F5F0FEF0BC0183048F40E9410115D
:1022F000F701E10FF11D80831F5FDD24DA94219641
:102300008881882321F0803211F08F32C9F6DD20D8
:1023100019F4C0E0D0E003C0888181112196CE017C
:10232000DF91CF911F910F91FF90EF90DF90089573
:10233000EC01F2CFCF92DF92FF920F931F93CF93D6
:10234000DF93EC016B018A01222321F0213009F097
:1023500049C02FC0FF248B858F708F3021F1CE01B3
:10236000B6014BE050E00E94EC2E0097E1F401151D
:10237000110521F0F801F4828B8585838C899D8974
:10238000A0E0B0E0AC01332722278A8D9B8DA0E02E
:10239000B0E0280F391F4A1F5B1F21153105410589
:1023A000510521F515C0F394F0E1FF16D9F0A09680
:1023B000D2CF90E08B858F708F3079F08881882321
:1023C00011F0853E51F40115110511F0F8019483C7
:1023D00021E030E040E050E009C09F5F903111F013
:1023E000A096E8CF20E030E040E050E0B901CA011B
:1023F000DF91CF911F910F91FF90DF90CF900895C3
:10240000DF92EF92FF920F931F93DF93CF93CDB79D
:10241000DEB72B970FB6F894DEBF0FBECDBF9C0181
:10242000D62E072F8BE0AE014F5F5F4FDA01E82F0A
:102430001D92EA95E9F7E62FF72FDF011D928A95A5
:10244000E9F7F90180818F3211F0A90103C0A901D8
:102450004F5F5F4F10E07E010894E11CF11C0BC040
:102460008D2D902F9C01D901F7018BE001900D92E9
:102470008150E1F71F5FCA01B7010E943E11AC0114
:10248000009771F7112311F480E001C08FEF2B96B4
:102490000FB6F894DEBF0FBECDBFCF91DF911F9175
:1024A0000F91FF90EF90DF900895CF92DF92EF921F
:1024B000FF920F931F93CF93DF936C017A018B01EF
:1024C000EC018E819F81A885B985E80EF91E0A1F4F
:1024D0001B1F4CA95DA97BA9EA0160E01BC0898193
:1024E00090E0FC01EE0FFF1FE80FF91F3196EE0F91
:1024F000FF1FEC0FFD1F858180FF09C08081918146
:10250000A281B3818E159F05A007B10731F06F5FDF
:10251000C65EDD4F671718F32DC0209759F1DE0115
:102520005A96F90180E092E001900D920197E1F74F
:10253000898190E0FC01EE0FFF1FE80FF91FEE0FFD
:10254000FF1FEC0FFD1F878182605CC0FA01818153
:1025500090E0FC01EE0FFF1FE80FF91F3196EE0F20
:10256000FF1FE40FF51F858180FF08C06F5F465E87
:102570005D4F01C060E0671748F347C04115510542
:1025800009F443C0DA015A96F90180E092E0019023
:102590000D920197E1F7DA0111968C9190E0FC0120
:1025A000EE0FFF1FE80FF91F3196EE0FFF1FE40F2C
:1025B000F51F86E0EF0119928A95E9F7DA011C927E
:1025C000E082F1820283138311968C91119790E03F
:1025D000FC01EE0FFF1FE80FF91FEE0FFF1FE40FC6
:1025E000F51F87818260878311968C9190E0FC01B2
:1025F000EE0FFF1FE80FF91FEE0FFF1FE40FF51F8F
:102600008781816087838FEF0DC0E6018881998182
:102610000296FC01A591B4918A819B81B801A70122
:10262000FD010995DF91CF911F910F91FF90EF90E0
:10263000DF90CF900895AF92BF92CF92DF92EF924A
:10264000FF920F931F93CF93DF938C016A017B015D
:10265000B22EA32EFC0186819781A085B185C80E7C
:10266000D91EEA1EFB1E44A955A963A99A01E901D6
:1026700020E01BC0898190E0FC01EE0FFF1FE80FF6
:10268000F91F3196EE0FFF1FEC0FFD1F858180FFB4
:1026900009C080819181A281B3818C159D05AE0511
:1026A000BF0531F02F5FC65EDD4F261718F316C049
:1026B000209719F513C0898190E0FC01EE0FFF1FF0
:1026C000E80FF91F3196EE0FFF1FEC0FFD1F8581FC
:1026D00080FF09C02F5FC65EDD4F02C0EA0120E027
:1026E000261748F323C0209709F1C801BE01A701AE
:1026F00096010E94F70F882369F08B2D9A2D9C017B
:10270000D901FE017A9680E092E001900D92019746
:10271000E1F71DC080E0DF91CF911F910F91FF90F5
:10272000EF90DF90CF90BF90AF900895F801808137
:102730009181FC01A591B491F80182819381B70147
:10274000A6012B2D3A2DFD010995882319F38FEF52
:10275000E2CF6F927F928F929F92AF92BF92CF9271
:10276000DF92EF92FF920F931F93CF93DF937C0141
:102770004A015B01622EDC01D4964D915C91D597A4
:10278000D396DC90EA0120E01BC0898190E0FC0137
:10279000EE0FFF1FE80FF91F3196EE0FFF1FEC0F32
:1027A000FD1F858180FF09C080819181A281B38155
:1027B00088159905AA05BB0531F02F5FC65EDD4F70
:1027C0002D1518F317C0209709F0F1C013C08981A7
:1027D00090E0FC01EE0FFF1FE80FF91F3196EE0F9E
:1027E000FF1FEC0FFD1F858180FF0EC02F5FC65EAF
:1027F000DD4F02C0EA0120E02D1548F3A0E06FEFA5
:1028000070E000E010E03EC08E01209709F057C054
:10281000A0E06FEF70E036C0FA018181282F30E030
:10282000C9010196FC01EE0FFF1FE80FF91FEE0F23
:10283000FF1FE40FF51F80818823F9F4F901EE0FE3
:10284000FF1FE20FF31F3196EE0FFF1FE40FF51F7E
:10285000858181FFECC0772351F00FC0FA018081A0
:10286000681758F0FA0180818A017FEF07C0FA01EA
:102870008081681710F08A0101C0862FAF5F465E25
:102880005D4F682FAD1540F2E8010115110599F073
:10289000898190E0FC01EE0FFF1FE80FF91F3196D0
:1028A000EE0FFF1FE00FF11F858181FF04C0C701FC
:1028B000B8010E943A0F0115110519F0E80189814C
:1028C0005EC0F70124A935A9D3A800E01FEF93E368
:1028D000792E8DE4C82E32C0D90111964C91443026
:1028E00040F5842F90E0FC01EE0FFF1FE80FF91F69
:1028F0003196EE0FFF1FE20FF31F858181FD02C0AD
:10290000E0E001C0EFE7D9018C91879DC00111245F
:102910006FEF70E00E94D82F4C9DC0011124969556
:10292000879596958795680F6E0F611710F4E901EA
:1029300001C0612F0F5F265E3D4F162F0D1560F20F
:10294000209709F462C0898190E0FC01EE0FFF1F1F
:10295000E80FF91F3196EE0FFF1FEC0FFD1F858169
:1029600081FF04C0C701BE010E943A0F89818430F3
:1029700020F08FED0E942F2448C08F5F898323E0D1
:10298000829FC00111240196880F991F8C0F9D1FF3
:10299000FC0186E0DF011D928A95E9F71882C701E4
:1029A000BE01A50194010E94F70F882371F161FE19
:1029B0000EC0898190E0FC01EE0FFF1FE80FF91FA8
:1029C000EE0FFF1FEC0FFD1F8781826087838981D7
:1029D00090E00196FC01EE0FFF1FE80FF91FEE0FCC
:1029E000FF1FEC0FFD1F80818F5F8083882311F410
:1029F0008FEF808388818F5F8883882311F48FEF26
:102A00008883BE01665E7F4F02C060E070E0CB014C
:102A1000DF91CF911F910F91FF90EF90DF90CF90BA
:102A2000BF90AF909F908F907F906F900895772385
:102A300009F418CF13CFFC01DB01CA01468157818D
:102A400060857185480F591F6A1F7B1FCF010E9447
:102A5000A9130895CF92DF92EF92FF920F931F93E5
:102A6000CF93DF93EC017A018B01B9018EA1803104
:102A700009F455C0803209F45EC08C3029F020E0A2
:102A800030E040E050E064C0A8019701337040702E
:102A90005070DA01C901880F991FAA1FBB1F820F4E
:102AA000931FA41FB51FB695A7959795879591700D
:102AB000FB01E80FF91FC0808F5F9140B1F4CE0198
:102AC000B801A7010E94A710AB01BC014F5F5F4F87
:102AD0006F4F7F4FCE0121E00E941B15FC01D0807B
:102AE000CE01BF010E943D1001C0D1808D2D90E02C
:102AF000E0FC05C08F709070982F882708C074E0A4
:102B0000880F991F7A95E1F7C2946FE0C6228C0D69
:102B1000911D9C01442737FD4095542F19C0F701A2
:102B2000F070EE0FFF1FE20FF31F808191819C0177
:102B300040E050E00DC0F701EF77F070EE0FFF1F9F
:102B4000EE0FFF1FE20FF31F20813181428153817D
:102B5000B901CA01DF91CF911F910F91FF90EF90C2
:102B6000DF90CF9008952F923F924F925F926F9295
:102B70007F928F929F92AF92BF92CF92DF92EF920D
:102B8000FF920F931F93DF93CF9300D000D000D01C
:102B9000CDB7DEB74C017E836D83FB014085518547
:102BA00062857385411551056105710509F4CDC034
:102BB0000E94A71069837A838B839C83C401498117
:102BC0005A816B817C8121E00E941B15382E292EB1
:102BD000ED81FE814085518562857385C401232D79
:102BE000322D0E942A15AB01BC01F40186A180316F
:102BF00071F08032A9F08C3009F098C0483FFFE0B6
:102C00005F07F0E06F07F0E07F0798F08FC0483F64
:102C10002FEF520720E0620720E0720750F086C0D5
:102C2000DB01CA01BF70885F9F4FAF4FBF4008F004
:102C30007DC0ED81FE8140875187628773878481E3
:102C40009581A681B7810196A11DB11D84839583CD
:102C5000A683B7832A013B01089441085108610803
:102C600071087A018B01AA24BB24650113C0C40139
:102C7000B801A701232D322D0E942A150894A11C0A
:102C8000B11CC11CD11C27013801AC01CB01DA01F8
:102C90007C018D01D801C7010197A109B1098415F3
:102CA0009505A605B70571F4C401B801A7010E94F6
:102CB000A71029813A814B815C81621773078407D1
:102CC0009507A9F2A114B104C104D10429F480E04C
:102CD00090E0A0E0B0E005C0D601C5010197A109D0
:102CE000B109ED81FE8180839183A283B383C40106
:102CF000632D722D0E943D108FEF26960FB6F8942B
:102D0000DEBF0FBECDBFCF91DF911F910F91FF901E
:102D1000EF90DF90CF90BF90AF909F908F907F907B
:102D20006F905F904F903F902F900895ED81FE81BE
:102D300080859185A285B385808B918BA28BB38B87
:102D4000C401632D722D0E943D1080E0D6CF0F93F9
:102D50001F93CF93DF938C01EB0188859985AA851A
:102D6000BB850097A105B10561F48C859D85AE8575
:102D7000BF8588879987AA87BB871C821D821E8290
:102D80001F8288899989AA89BB890097A105B10505
:102D900009F126C08C819D81AE81BF812881398156
:102DA0004A815B81820F931FA41FB51F8C839D8373
:102DB000AE83BF8388859985AA85BB85820F931FC3
:102DC000A41FB51F88879987AA87BB871882198295
:102DD0001A821B82C801BE010E94B3158823D1F656
:102DE000688979898A899B89DF91CF911F910F9199
:102DF0000895CF92DF92EF92FF920F931F93CF939C
:102E0000DF936C01EB0179018A018C819D81AE8198
:102E1000BF81281739074A075B0740F088859985E5
:102E2000AA85BB850097A105B10581F41C821D828E
:102E30001E821F828C859D85AE85BF858887998778
:102E4000AA87BB87188219821A821B828C819D8176
:102E5000AE81BF818E159F05A007B10799F129C0EA
:102E600088819981AA81BB810097A105B105D9F01C
:102E70000197A109B10988839983AA83BB832F5F36
:102E80003F4F4F4F5F4F2C833D834E835F83888539
:102E90009985AA85BB850196A11DB11D8887998753
:102EA000AA87BB8706C0C601BE010E94B31588234E
:102EB00051F02C813D814E815F812E153F054007E9
:102EC000510771F68FEFDF91CF911F910F91FF9016
:102ED000EF90DF90CF9008952F923F924F925F92A4
:102EE0006F927F928F929F92AF92BF92CF92DF921A
:102EF000EF92FF920F931F93DF93CF93CDB7DEB77F
:102F0000A4970FB6F894DEBF0FBECDBF1C017F8F14
:102F10006E8F19A308A3EAA2FE01319688E1DF01B2
:102F20001D928A95E9F729873A874B875C872D8719
:102F30003E874F87588B223031054105510540F0BF
:102F400020E030E040E050E0CF01EBA39CA3A4C020
:102F5000F10186A18C3019F0803109F0AEC0D101A9
:102F60009796AD90BD90CD90DC909A9754968D91A8
:102F70009C915597F5E096958795FA95E1F73C0178
:102F8000882499246A0C7B1C8C1C9D1C29C0C101BF
:102F9000B601A50121E00E941B152C016E8D7F8DCD
:102FA00048A159A12AA10E949A117B018C016115A7
:102FB00071058105910559F0E8A1F9A1309721F03B
:102FC000A082B182C282D382C101B20150C0C101CC
:102FD000B2010E943D100894A11CB11CC11CD11C5F
:102FE000A614B704C804D90490F267C049845A846F
:102FF0006B847C841D8E46C0C101B301A2010E9476
:10300000E60EAB01BC01BD8DAB2EBB24CC24DD2470
:103010004A0D5B1D6C1D7D1DC10121E00E941B1529
:10302000982E892E6E8D7F8D48A159A12AA10E94CC
:103030009A117B018C016115710581059105D1F013
:10304000E8A1F9A1EF2B81F0C101B301A2010E9417
:10305000E60EA60EB71EC81ED91EA8A1B9A1AD9234
:10306000BD92CD92DC921397C101692D782D0E94FB
:103070003D1026C0C101692D782D0E943D10BD8DE7
:10308000BF5FBD8FF1018089FD8DF81708F4B4CFC3
:10309000298D3A8D4B8D5C8DDA01C9010196A11DF8
:1030A000B11D898F9A8FAB8FBC8FC1016BA17CA1A1
:1030B0000E94F916882309F099CFEE24FF24870196
:1030C000B701C801A4960FB6F894DEBF0FBECDBFFE
:1030D000CF91DF911F910F91FF90EF90DF90CF90F4
:1030E000BF90AF909F908F907F906F905F904F9028
:1030F0003F902F9008952F923F924F925F926F9240
:103100007F928F929F92AF92BF92CF92DF92EF9277
:10311000FF920F931F93DF93CF93CDB7DEB72E9718
:103120000FB6F894DEBF0FBECDBF2C01FB015E874A
:103130004D87490180818F3201F5D20196968C919D
:10314000803231F0A1E0AA2EB12CC12CD12C07C0C5
:10315000D2015696AD90BD90CD90DC9059973196A6
:103160008114910431F0D401AD92BD92CD92DC92E4
:1031700013978081882389F471C0D2019B96AD900A
:10318000BD90CD90DC909E972115310531F0D9018D
:10319000AD92BD92CD92DC921397FF241C861E0146
:1031A0000894211C311C45C0C201B101A601950142
:1031B0000D851E85EE240E946C179B01AC016115E4
:1031C00071058105910539F4C301B1010E943E11D9
:1031D000892B01F545C0AD85BE8515968C9184FF80
:1031E00013C08114910429F0F401208331834283B8
:1031F0005383FF2031F0D4011D921D921D921C9229
:10320000139759016A0111C0C301B1010E943E1117
:10321000892B49F08114910419F1F4011082118273
:10322000128213821DC0FF24FA94FC85FF5FFC8785
:10323000F301CF01B1010E943E113C01009709F05A
:10324000B3CF8C85882361F0AD85BE8515968C91B2
:1032500084FD04C0FF2011F081E003C082E001C0C2
:1032600080E02E960FB6F894DEBF0FBECDBFCF9193
:10327000DF911F910F91FF90EF90DF90CF90BF9063
:10328000AF909F908F907F906F905F904F903F9006
:103290002F900895EF92FF920F931F93CF93DF9398
:1032A000EC01F62EE72E8A01FA01408151816281FC
:1032B000738122E00E941B15BC01F8018481E82F74
:1032C000F0E0B5E0EE0FFF1FBA95E1F7E60FF71F4C
:1032D0002F2D3E2DC901DC0180E20D90019281501D
:1032E000E1F7CE010E943D10DF91CF911F910F9128
:1032F000FF90EF9008952F923F924F925F926F92BE
:103300007F928F929F92AF92BF92CF92DF92EF9275
:10331000FF920F931F93DF93CF9300D000D0CDB7D0
:10332000DEB79C838B83FC0167A470A881A892A858
:10333000F2E06F1671048104910450F0FC0182A147
:1033400093A1A4A1B5A186159705A805B90528F4F0
:1033500092E0692E712C812C912C84017301AA2496
:10336000BB2465011A82198202C0620151018B815E
:103370009C81B801A7010E94A7101B012C016A15AE
:103380007B058C059D0599F089819A81892B31F007
:103390008B819C8169817A810E943D108B819C8107
:1033A000B201A10121E00E941B159A8389838B81C0
:1033B0009C81B801A70129813A810E942A156115D3
:1033C000710581059105F9F00894E11CF11C011DBE
:1033D000111DEB81FC8182A193A1A4A1B5A18E1541
:1033E0009F05A007B10728F482E0E82EF12C012DFB
:1033F000112DE614F7040805190509F0B6CFEE24DF
:10340000FF24870106C0E114F1040105110509F448
:10341000ACCF89819A81892B31F08B819C81698124
:103420007A810E943D10EB81FC81E7A6F0AA01ABF6
:1034300012ABB701C8010F900F900F900F90CF9172
:10344000DF911F910F91FF90EF90DF90CF90BF9091
:10345000AF909F908F907F906F905F904F903F9034
:103460002F9008954F925F926F927F928F929F92CA
:10347000AF92BF92CF92DF92EF92FF920F931F9382
:10348000CF93DF932C013A014B01580169010E944F
:10349000A7107B018C01F20181899289A0E0B0E044
:1034A000A8019701281B390B4A0B5B0B828D938D6A
:1034B000A48DB58D281739074A075B0708F0B8C0F7
:1034C000E114F1040105110509F4B2C0C201B8010B
:1034D000A70122E00E941B15EC01F20186A18031B8
:1034E00009F48CC0803209F492C08C3009F09CC081
:1034F000A4019301337040705070DA01C901880F44
:10350000991FAA1FBB1F820F931FA41FB51FB6953B
:10351000A795979587959170E1E0EE2EF12C012DFE
:10352000112DE620F72008211921F1E08F3F9F0798
:10353000E9F5FE01E150FE4FE114F104010511052A
:1035400011F4A08207C080818F709A2D9295907F90
:10355000890F8083C201B401A3010E94A710AB01AF
:10356000BC014F5F5F4F6F4F7F4FC20122E00E944F
:103570001B15FC01E114F1040105110551F4208132
:10358000207FBB27AD2D9C2D8B2D8F70280F208386
:1035900008C064E0D694C794B794A7946A95D1F70D
:1035A000A082C201BF010E943D103EC0DE01A80FF3
:1035B000B91FE114F1040105110579F4AC92FC0185
:1035C0003196EC0FFD1F2081207FBB27AD2D9C2D58
:1035D0008B2D8F70280F208327C08C918F709A2D90
:1035E0009295907F890F8C9344E0D694C794B794BA
:1035F000A7944A95D1F71196AC9216C0F301F070DA
:10360000EE0FFF1FEC0FFD1FB182A0820DC0F30172
:10361000EF77F070EE0FFF1FEE0FFF1FEC0FFD1F97
:10362000A082B182C282D382C201BE010E943D103B
:10363000DF91CF911F910F91FF90EF90DF90CF908E
:10364000BF90AF909F908F907F906F905F904F90C2
:1036500008952F923F924F925F926F927F928F9236
:103660009F92AF92BF92CF92DF92EF92FF920F9311
:103670001F93DF93CF9300D000D000D0CDB7DEB73B
:103680009E838D833B0119012A01FB018485958569
:10369000A685B7850297A105B10508F47CC08D8188
:1036A0009E810E94A71669837A838B839C83ED8118
:1036B000FE8167A770AB8B8181AB92AB5201410158
:1036C00052C08D819E810E947B196B017C01611526
:1036D000710581059105F1F48D819E810E94F110A3
:1036E0008B019C018D819E8149815A816B817C81F6
:1036F0000E94321A8981F301808B8A81818B8B81B0
:10370000828B8C81838B281439044A045B0409F072
:1037100044C041C08D819E8149815A816B817C81E9
:10372000970186010E94321A089481089108A10825
:10373000B10881149104A104B10489F48D819E81A2
:103740000E94F1108B019C018D819E81B701A60121
:103750000E94321AF301C08AD18AE28AF38AC982AE
:10376000DA82EB82FC8281149104A104B10409F095
:10377000A8CFF30184899589A689B7890097A10507
:10378000B10559F0820D931DA41DB51D848B958B39
:10379000A68BB78B02C080E001C08FEF26960FB6D4
:1037A000F894DEBF0FBECDBFCF91DF911F910F9177
:1037B000FF90EF90DF90CF90BF90AF909F908F9051
:1037C0007F906F905F904F903F902F900895BF92A1
:1037D000CF92DF92EF92FF920F931F93CF93DF93DD
:1037E000EC010E94E60EB62E262F372FAC01C90140
:1037F000DA017C018D01C12C82E0D82E14C0CE01EB
:10380000B801A70122E00E941B15BC01DC01C60122
:103810001D920197E9F7CE010E943D100894E11C2A
:10382000F11C011D111D9E2D9B198889981738F3D5
:10383000DF91CF911F910F91FF90EF90DF90CF908C
:10384000BF9008958F929F92AF92BF92CF92DF92D6
:10385000EF920F931F93DF93CF93CDB7DEB7A79768
:103860000FB6F894DEBF0FBECDBF6C018B015A01BD
:1038700019821A821B821C829E012F5F3F4F0E9479
:103880007B18882309F051C095E0892E912C8C0E6D
:103890009D1EC801B4010E940012882309F445C08E
:1038A00029813A814B815C81C601B4018501EE24F6
:1038B000E3940E946C176115710581059105B9F5B6
:1038C00089819A81AB81BC818E01005F1F4F28E105
:1038D000F80111922A95E9F7888F998FAA8FBB8FEB
:1038E0008C8F9D8FAE8FBF8FC601B80121E030E075
:1038F00040E050E00E94291B8823B9F0C601B801BE
:103900000E94A716AB01BC01C6010E94E71B2981DA
:103910003A814B815C81C601B40185010E946C171C
:10392000611571058105910511F480E001C08FEFEB
:10393000A7960FB6F894DEBF0FBECDBFCF91DF9133
:103940001F910F91EF90DF90CF90BF90AF909F901D
:103950008F9008952F923F924F925F926F927F9235
:103960008F929F92AF92BF92CF92DF92EF92FF928F
:103970000F931F93DF93CF9300D000D0CDB7DEB766
:103980001C01DC0150968C9144245524320188247A
:1039900099245401282F30E040E050E029833A83F5
:1039A0004B835C8348C0C101B501A4010E94A710EC
:1039B0007B018C01D10151968D919C915297A0E091
:1039C000B0E0A8019701281B390B4A0B5B0BF101F2
:1039D000828D938DA48DB58D281739074A075B0713
:1039E000E8F4E114F10401051105C1F0C101B801C9
:1039F000A70121E00E941B156C01C101B501A401C2
:103A000096010E942A157B018C01C101B6010E941A
:103A10003D10E114F1040105110541F429813A81B9
:103A20004B815C81420E531E641E751E0894811CDE
:103A3000911CA11CB11CF10182A193A1A4A1B5A16B
:103A400088169906AA06BB0608F4ADCFA301920119
:103A50005695479537952795B901CA010F900F9054
:103A60000F900F90CF91DF911F910F91FF90EF90EA
:103A7000DF90CF90BF90AF909F908F907F906F908E
:103A80005F904F903F902F9008953F924F925F929A
:103A90006F927F928F929F92AF92BF92CF92DF925E
:103AA000EF92FF920F931F93CF93DF93EC01598313
:103AB00048833B832A831D828CA99DA9892B49F4C5
:103AC0006BAB862F90E06AE172E00E94BD2D8CAB5B
:103AD0009DABCE0140E050E060E070E021E00E944C
:103AE000A9138C01009711F480E08AC1FC01EE500B
:103AF000FE4F33249C012E543E4F8081813051F083
:103B0000843041F0863031F08B3021F08C3511F06B
:103B10008E3599F48D8384819581A681B7818E83BA
:103B20009F83A887B98780859185A285B3858A8779
:103B30009B87AC87BD8733243A947097E217F307CD
:103B4000E1F63320B9F4288139818BE08D831E8220
:103B50001F82188619862C5F3F4FF90145915491B9
:103B60008A819B81FA0109956A877B878C879D876B
:103B700033243A94CE01B8010E943D10CE0140E0BA
:103B800050E060E070E021E00E941B15BC018C0158
:103B9000DC011B968D919C911C979F878E87FB0162
:103BA0008585888B1E968D919C911F979A8B898B0A
:103BB00080898B8B51968D919C9152979D8B8C8B8C
:103BC00084A595A5A6A5B7A58E8B9F8BA88FB98F29
:103BD000DB0156966D907C905797C4A0D5A0E6A0C7
:103BE000F7A053964D905C90549780A091A0A2A00E
:103BF000B3A0CE010E943D1002501E4FF8018081FB
:103C0000918185559A4A09F0F9C08E859F8580502B
:103C1000924009F0F3C0488920E030E0403111F4CF
:103C200021E030E080E090E0483011F481E090E065
:103C3000282B392B80E090E0403211F481E090E0B5
:103C4000282B392B80E090E0403411F481E090E0A3
:103C5000282B392B90E0842F8150823008F491E09A
:103C600080E0443009F481E0982B892F90E0282BE4
:103C7000392B232B09F4C2C089899A89892B09F42D
:103C8000BDC06114710419F06301EE24FF24CA8ED3
:103C9000DB8EEC8EFD8E8A859B85AC85BD858C1573
:103CA0009D05AE05BF0508F4A9C04114510419F0E3
:103CB0004201AA24BB248E8E9F8EA8A2B9A2CE84D4
:103CC000DF846B8970E080E090E02A8D3B8D4C8D25
:103CD0005D8D0E94B92F7B018C0110950095F094A9
:103CE000E094E11CF11C011D111D89899A89A0E055
:103CF000B0E0E81AF90A0A0B1B0BC60101972C89E0
:103D00003D8975E0220F331F7A95E1F7820F931FEB
:103D1000B6010E94D82F80E090E0E61AF70A080B5F
:103D2000190BE80CF91C0A1D1B1D288930E040E026
:103D300050E0C801B7010E94EC2FC901DA018AA343
:103D40009BA3ACA3BDA3853FEFE09E07E0E0AE07D9
:103D5000E0E0BE0710F48CE006C0855F9F4FA040F6
:103D6000B04038F480E18EA31E8A1F8A188E198E07
:103D700002C080E28EA36B8970E080E090E02A8D23
:103D80003B8D4C8D5D8D0E94B92F7B018C01898903
:103D90009A89A0E0B0E0E80EF91E0A1F1B1FEFA2EF
:103DA000F8A609A71AA78EA18032B1F4688970E03D
:103DB00080E090E02E893F89488D598D2250304017
:103DC000404050400E94B92FE60EF71E081F191FF1
:103DD000EFA2F8A609A71AA78EA1803229F081E0E8
:103DE00090E0A0E0B0E004C08E899F89A88DB98DD5
:103DF0008BA79CA7ADA7BEA78FEF01C080E0832152
:103E00008C83DF91CF911F910F91FF90EF90DF9006
:103E1000CF90BF90AF909F908F907F906F905F906A
:103E20004F903F900895FC0161857285838594854C
:103E3000089589EF96E00895BF92CF92DF92EF92B6
:103E4000FF920F931F93B82EC92E0E940F0C7B0177
:103E50008C018B2D9C2D0E94AC278B2D9C2D0E94BC
:103E6000AC27D82E8FEFD81651F0C801B70120E249
:103E700031EA47E050E00E946E23882371F38D2DD4
:103E80001F910F91FF90EF90DF90CF90BF9008951A
:103E90000F931F938C0160E00E945926C8010E9475
:103EA000AC271F910F910895BF92CF92DF92EF92AE
:103EB000FF920F931F93DF93CF9300D000D000D0D9
:103EC000CDB7DEB7C82EB92ED62E79018A0167FF8D
:103ED0000CC067E720E030E040E050E00E94541F53
:103EE000823008F051C08FE7D8228C2D9B2D0E9484
:103EF000481F80E4D81639F48C2D9B2D6FEF0E945B
:103F0000592625E917C08C2D9B2D6FEF0E9459264D
:103F10008C2D9B2D0E941C1F8F3F31F08C2D9B2DD3
:103F20000E94481F8FEF30C088E4D81611F427E8AC
:103F300001C021E0D982812F9927AA27BB278A8334
:103F4000C801AA27BB278B83BB27A12F902F8F2DBA
:103F50008C83ED822E838C2D9B2DBE016F5F7F4F56
:103F600046E050E00E94B5268CE4D81621F48C2D52
:103F70009B2D0E94AC271AE08C2D9B2D0E94AC2714
:103F800087FF02C01150C1F726960FB6F894DEBF26
:103F90000FBECDBFCF91DF911F910F91FF90EF909A
:103FA000DF90CF90BF900895FF920F931F93CF9310
:103FB000DF93182F092FEB01F42E0E941C1F8F3F57
:103FC000E1F4812F902F6F2D0E94B1278DEFF8160D
:103FD000B1F0812F902FBE0140E052E00E94B52643
:103FE000812F902F6FEF7FEF0E94B427812F902FAA
:103FF0000E94AC278F71853011F080E001C08FEFF7
:10400000DF91CF911F910F91FF900895BF92CF92B2
:10401000DF92EF92FF920F931F93CF93DF93EC0108
:104020006901B02E8885882309F45AC0002309F459
:1040300059C02115310509F457C08D8590E083FFE3
:1040400003C07A018B0109C07A018B0149E0EE0CB3
:10405000FF1C001F111F4A95D1F721E0B21689F409
:10406000CE0168E5A80197010E94541F8823A9F595
:10407000CE01B6014EEF0E94D41F882371F1BB24FC
:104080002CC086709070892B41F02B2D30E040E0E1
:1040900050E0CE0167ED0E94541FCE0169E5A801F2
:1040A00097010E94541F8823C1F4CE01B6014CEF42
:1040B0000E94D41F882339F0BA9429F080E092E05E
:1040C000C80ED91EF2CFCE0160E070E04DEF0E9425
:1040D000D41F882311F4BB24B394CE010E94481F3F
:1040E000BB2011F48FEF01C080E0DF91CF911F91D1
:1040F0000F91FF90EF90DF90CF90BF9008950F93B6
:1041000001E00E9406200F910895AF92BF92CF92D6
:10411000DF92EF92FF920F931F93CF93DF93D82EEE
:10412000C92EEB015A010E940F0C7B018C018D2DD1
:104130009C2D0E94AC278E3F51F0C801B70120E4AE
:104140003DE043E050E00E946E23882381F38D2DF3
:104150009C2DBE01A5010E9407278D2D9C2D0E943C
:10416000A1278FEFDF91CF911F910F91FF90EF90DB
:10417000DF90CF90BF90AF900895EF92FF920F9392
:10418000CF93DF93EC0179018885882309F448C037
:10419000002309F447C02115310509F445C08D8578
:1041A00083FF03C09A01AB0109C09A01AB0169E02A
:1041B000220F331F441F551F6A95D1F7013081F438
:1041C000CE0161E50E94541F882339F5CE01B70165
:1041D00040E052E00E9485208823F9F000E01DC0F5
:1041E000CE0162E50E94541F8823B9F4CE01B701C5
:1041F00040E052E00E948520882339F0015029F0E8
:1042000080E092E0E80EF91EF1CFCE016CE420E0F0
:1042100030E040E050E00E94541FCE010E94481F51
:10422000002311F48FEF01C080E0DF91CF910F9157
:10423000FF90EF9008950F9301E00E94BD200F9131
:1042400008954F925F926F927F928F929F92AF925A
:10425000BF92CF92DF92EF92FF920F931F93DF9363
:10426000CF93CDB7DEB764970FB6F894DEBF0FBE1D
:10427000CDBF7C012C0114E6C2010E94AC27115075
:10428000D9F7DE2CCF2CC7016FEF0E94592600E032
:1042900012E0C2010E94AC2701501040D1F78D2DD1
:1042A0009C2D60E00E94592600E010E0C70160E408
:1042B00020E030E040E050E00E94541F813009F4DB
:1042C0000EC10F5F1F4F8FEF0F3F180779F7E4C044
:1042D000C2010E94AC27F80181938F01E615F70512
:1042E000B9F78B81813009F0D7C08C818A3A09F007
:1042F000D3C0C601B50120E432E44FE050E00E9493
:104300006E23882351F4C70169EE20E030E040E0DD
:1043100050E40E94541F882361F7C601B50120E4D0
:1043200032E44FE050E00E946E23882309F0B4C0CD
:10433000C7016AE720E030E040E050E00E94541FEF
:10434000882309F0A9C0C2010E94AC27F40181931F
:104350004F01E017F107B9F7898186FDDAC004E063
:10436000D9C0C70169EE20E030E040E050E00E9493
:10437000541F823018F011E401E002C019EE02E08F
:10438000C601B50120E432E44FE050E00E946E2304
:10439000882351F4C701612F20E030E040E050E075
:1043A0000E94541F882361F7C601B50120E432E45E
:1043B0004FE050E00E946E23882309F06DC0C701D2
:1043C00060E520E032E040E050E00E94541F882386
:1043D00009F062C09FC0C701BE016B5F7F4F40E123
:1043E00050E00E948520882309F44CC08D8182957D
:1043F000869586958370EE854D85813099F42E2FB4
:1044000030E02F5F3F4F942F80E0280F391FA90124
:1044100060E070E0BAE0440F551F661F771FBA9541
:10442000D1F734C042954695469543702C8530E0CF
:10443000220F331F220F331F240F311D2F5F3F4FD9
:104440008B8590E083709070982F8827990F990F33
:10445000280F391FA90160E070E08A858F702F85D1
:10446000221F2227221F820F8E5FE370EE0F8E0F16
:1044700090E0099704C0440F551F661F771F8A9567
:10448000D2F704C040E050E060E070E0F7014187FF
:1044900052876387748701C000E0C7010E94481FEC
:1044A000002311F08FEF01C080E0F70105878087BE
:1044B00064960FB6F894DEBF0FBECDBFCF91DF91EB
:1044C0001F910F91FF90EF90DF90CF90BF90AF9032
:1044D0009F908F907F906F905F904F9008950E9473
:1044E0000F0C5B016C01C70168E42AEA31E040E08F
:1044F00050E00E94541F813009F033CF4E010894E0
:10450000811C911C840175E0672E712C6C0E7D1E40
:10451000DFCE0CE0C70169E420E030E040E050E08D
:104520000E94541F882309F0ADCF55CFEAE7F0E091
:104530008081877F808380818F7780830895EAE7F9
:10454000F0E090818770987F892B80830895982F61
:1045500085FF04C080917B00886003C080917B0050
:10456000877F80937B0080917C009F71807E892B68
:1045700080937C001092DA0480917A0080618093AD
:104580007A0080917A00806480937A0080917A002A
:1045900086FDFCCF2091780030917900C901089503
:1045A0000E94A722969587959695879508951F92C4
:1045B0000F920FB60F9211248F938FEF8093DA042E
:1045C0008F910F900FBE0F901F901895EF92FF9252
:1045D0000F931F93CF93DF9380917A00806880932D
:1045E0007A0080917A008F7D80937A0080917A00A2
:1045F000887F866080937A0080917C008F738064CE
:1046000080937C0080917C008F7D80937C008091E2
:104610007A00886080937A008FEF8093DA04789430
:1046200080914902C82FD0E0219700E010E07E0180
:104630000FC0C701801B910B089724F09E01285ED4
:10464000822F01C08C2F0E94A72221970F5F1F4F3E
:104650003FEFCF3FD30769F7DF91CF911F910F91C4
:10466000FF90EF9008951F93CF93DF93EC01162FE7
:1046700061380CF411E8E881F981309779F02591DF
:1046800034912115310551F08B8181FD02C0612FDC
:1046900002C0612F6195CE01F90109951A83DF915E
:1046A000CF911F910895DC01962F917013968C91F4
:1046B00013978E7F892B13968C9313978D919C91D2
:1046C0001197009751F0FC013296259134912115F4
:1046D000310519F0CD01F901099508950F931F9344
:1046E00000E010E00E9477231F910F9108958F92B0
:1046F0009F92AF92BF92CF92DF92EF92FF920F9371
:104700001F93CF93DF936B017C0149015A01E801AC
:104710000E940F0C6C197D098E099F096815790597
:104720008A059B0568F00115110541F068197909A2
:104730008A099B09688379838A839B838FEF0CC0E6
:104740000115110541F0861A970AA80AB90A88824C
:104750009982AA82BB8280E0DF91CF911F910F9155
:10476000FF90EF90DF90CF90BF90AF909F908F9091
:10477000089528EE33E040E050E00E94B92F0E94F7
:10478000C2230895AF92BF92CF92DF92EF92FF9231
:104790000F931F935B016C010E940F0C7B018C0136
:1047A00001C000000E940F0C6E197F09800B910B55
:1047B0006A157B058C059D05A0F31F910F91FF9055
:1047C000EF90DF90CF90BF90AF9008954F925F929F
:1047D0006F927F928F929F92AF92BF92CF92DF9211
:1047E000EF92FF920F931F932B015A013901780129
:1047F000E21AF30A00E010E09C01261B370B442765
:1048000037FD4095542FC801B7010E94B92FA41855
:10481000B508CC24B7FCC094DC2CA60195010E94FD
:104820000E3088249924260D371D481D591DC901B5
:104830001F910F91FF90EF90DF90CF90BF90AF90BE
:104840009F908F907F906F905F904F900895809190
:10485000DB0408959093DF048093DE0408951F9392
:10486000182F8091DB04882309F050C01093DB04DB
:104870008091E0049091E104009749F00E949D240A
:10488000882329F080EE94E060E00E94002580916A
:10489000EB049091EC040097C9F1212F332727FDF9
:1048A000309517FF17C000D000D000D0EDB7FEB78D
:1048B0003196ADB7BEB712969C938E9311978EE04A
:1048C00097E09383828388279927821B930B958394
:1048D000848312C000D000D000D0EDB7FEB731966F
:1048E000ADB7BEB712969C938E9311978FEF96E05B
:1048F00093838283358324830E94002F8DB79EB7D4
:1049000006960FB6F8949EBF0FBE8DBF1F910895F7
:104910009C01009781F0FC01859194910496FC0123
:10492000A591B4912E5F3F4FF90194918C91892309
:1049300011F08FEF089580E008959C01009781F0B9
:10494000FC01859194910296FC01A591B4912E5F92
:104950003F4FF90194918C91892311F08FEF0895C5
:1049600080E00895CF93DF939C010097F9F0FC015C
:1049700045915491CA010296FC01A591B491FA01A6
:10498000C591D4912E5F3F4FF90194913FB7F894B0
:104990008C91292F209582238C93662319F088818E
:1049A000892B02C08881822388833FBFDF91CF910A
:1049B0000895CF93DF939C010097F9F0FC01459196
:1049C0005491CA010296FC01C591D491FA01A591B6
:1049D000B4912E5F3F4FF90124913FB7F8946623BD
:1049E00019F08C91822B04C08C91922F9095892381
:1049F0008C938881822B88833FBFDF91CF9108956C
:104A00001F93CF93DF93EC01162F88819981009734
:104A1000A9F03A8130FD05C020E0662309F421E0C9
:104A2000122F31FD06C0612F0E94D9248A81826035
:104A30008A8388819981612F0E94312CDF91CF91E7
:104A40001F9108950E94EC0C0E94960C0E942C0C61
:104A500078940E94070D0E942E0B0E940F0C609309
:104A60001B0470931C0480931D0490931E040E94E9
:104A7000370B60931F04709320048093210490935C
:104A8000220478940E94DD2B80911F0490912004D1
:104A9000A0912104B09122040097A105B10519F459
:104AA00016C00E94DD2B60911B0470911C04809144
:104AB0001D0490911E0420911F0430912004409108
:104AC0002104509122040E946E23882351F30E94F6
:104AD0000F0C9B01AC0160931B0470931C0480932A
:104AE0001D0490931E046091170470911804809126
:104AF000190490911A046F5F7F4F8F4F9F4F6093FF
:104B00001704709318048093190490931A040E9458
:104B1000960BAFCF90E008954FB7F8942091D10253
:104B20003091D2029093D2028093D1024FBFC9013B
:104B300008951F93182F8A3031F4E091D102F0913B
:104B4000D2028DE00995E091D102F091D202812F3D
:104B500009951F9108958AE00E94992508958FEF85
:104B60009FEF0895DF93CF93CDB7DEB76E817F813E
:104B70009E01285F3F4F8D81813031F483ED92E0BB
:104B8000A9010E944A2F05C083ED92E0A9010E946D
:104B90007D2CCF91DF9108950E9499250895CF93A0
:104BA000DF93EC01009769F08985882351F08881B3
:104BB00099810296FC0125913491CE01F901099564
:104BC0001986DF91CF910895DC01009769F017965F
:104BD0006C9317978D919C9111970896FC012591E4
:104BE0003491CD01F90109950895DC01009769F030
:104BF00018966C9318978D919C9111970696FC01CD
:104C000025913491CD01F90109950895DC010097B2
:104C100069F016966C9316978D919C911197049656
:104C2000FC0125913491CD01F90109950895DF9298
:104C3000EF92FF920F931F93CF93DF93EC01D62E49
:104C4000009779F18985882361F5E881F981E590FC
:104C5000F49000E010E018C0C801880F991F2A8165
:104C60003B81280F391FF901A591B4911196DC936E
:104C7000CE9314968D919C911597009719F06FEF34
:104C80000E94D9240F5F1F4F8C819D81081719073F
:104C900018F31B861A86CE016D2DF70109958FEF4B
:104CA0008987DF91CF911F910F91FF90EF90DF9057
:104CB0000895EF92FF920F931F93CF93DF938C0190
:104CC000FC01C081D181209709F445C0E881F981B8
:104CD0007096E590F490662341F18A859B85009754
:104CE00019F060E00E945926F80162818F818617D1
:104CF00019F0CE010E94E425F801638188858617AA
:104D000019F0CE010E94F525E114F10421F0C8014B
:104D10006FEFF70109951B870A87F8018481958158
:104D20000097E1F00E94E82B19C0FC018481958175
:104D3000009711F00E940D2C8A859B8580179107A2
:104D400069F41B861A86E114F10441F0C80160E0A1
:104D5000F701099503C082EE0E942F24DF91CF91C5
:104D60001F910F91FF90EF900895AF92BF92CF9255
:104D7000DF92EF92FF920F931F93CF93DF93EC019B
:104D8000B62EA72E7A0141155105B1F1088119817E
:104D90000115110571F1F801828593858C179D0726
:104DA00021F0CE016FEF0E945926F8018081918198
:104DB000FC013E96259134912115310539F0CE0143
:104DC0006B2D7A2DA701F901099516C0FC013A96C1
:104DD000C590D4908B2D9A2D9C01E9016991C80151
:104DE000F60109950894E108F108E114F104B1F71E
:104DF00003C082EE0E942F24DF91CF911F910F916B
:104E0000FF90EF90DF90CF90BF90AF9008958F927A
:104E10009F92AF92BF92CF92DF92EF92FF920F9349
:104E20001F93CF93DF937C01962E872E6A01411545
:104E3000510509F439C0FC010081118101151105EA
:104E400081F1F801828593858E159F0521F0C701B8
:104E50006FEF0E945926F80180819181FC013C96F8
:104E6000259134912115310539F0C701692D782D2F
:104E7000A601F901099518C0FC013A96A590B490D5
:104E8000892D982D9C01E901C801F7016781F50181
:104E9000099589930894C108D108C114D104A1F7D8
:104EA00003C082EE0E942F24DF91CF911F910F91BA
:104EB000FF90EF90DF90CF90BF90AF909F908F903A
:104EC00008951F93CF93DF93FC01162FC081D181EA
:104ED0002097A1F08A859B858E179F0721F0CF012F
:104EE0006FEF0E945926888199810A96FC012591CD
:104EF0003491CE01612FF901099504C082EE0E9420
:104F00002F2480E0DF91CF911F910895DF92EF92DF
:104F1000FF920F931F937C01D62E672F0E9461276B
:104F2000182F00E0C7016D2D0E946127282F30E067
:104F3000202B312BC9011F910F91FF90EF90DF9033
:104F40000895FC01878190E0782F6627682B792BE4
:104F5000CF010E9486270895FC0167810E94612786
:104F600008950E9461270895FF920F931F938C016B
:104F7000F62E672F0E946127C8016F2D0E946127BE
:104F80001F910F91FF9008958CB58F7B8CBD089574
:104F9000662319F48CB58F7D02C08CB580628CBD00
:104FA0000895613051F0613028F0623061F0633073
:104FB000B9F410C08CB5877F08C08CB5877F8CBDD5
:104FC0008CB5846005C08CB588608CBD8CB58B7F3A
:104FD0008CBD08958CB588608CBD8CB584608CBD0B
:104FE00008958CB58D7F8CBD8CB58E7F8CBD8DB5B5
:104FF0008E7F8DBD6031A9F0613128F4623051F0AF
:105000006830F9F40BC0603491F06038A1F0603280
:10501000C1F40AC08DB581608DBD08958DB58160E4
:105020008DBD8CB5816005C08DB581608DBD8CB5A1
:1050300082608CBD08958CB581608CBD8CB582601A
:105040008CBD0895FF920F931F93DF93CF930F9220
:10505000CDB7DEB78C01FFB6F894662339F0219AFC
:10506000229A23982B9A209A80E502C0239A80E402
:105070008CBDC801F80166810E94F127F801808586
:10508000882319F48CB58F7D02C08CB580628CBDED
:10509000C801F80167810E94D1278DB589838EB53B
:1050A0008983FFBE0F90CF91DF911F910F91FF90E9
:1050B00008956EBD0DB407FEFDCF8EB50895BF9265
:1050C000CF92DF92EF92FF920F931F93CF93DF93D4
:1050D0006C01B0900F022CE935E090E0C0E0D0E028
:1050E0002DC0285F3F4FF901E49028503040F9016E
:1050F00077962A5F3F4F80E0A0E0B0E005911491E1
:10510000F901F4902650304014C0B8016A0F7B1F9B
:10511000FB013E96459154914115510541F04C15C6
:105120005D0529F4FF2011F0EB010AC0EB018F5F50
:1051300050968E1550F39F5F245D3F4F9B1588F26C
:10514000CE01DF91CF911F910F91FF90EF90DF90F3
:10515000CF90BF9008959C010B96FC01A591B4914E
:10516000235F3F4FF901249170E0022E02C0660FC9
:10517000771F0A94E2F781E090E002C0880F991F40
:105180002A95E2F7282F220F282B9C91822F862325
:1051900020952923822B8C930895CF93DF939C0134
:1051A0002E5F3F4FF9018491225030409CE2899F4D
:1051B000A001112444565A4F485F5F4FFA01849171
:1051C000485050408823C1F0C9010696FC01C591A2
:1051D000D491FA013696E491EE2319F0798368832D
:1051E0000EC06F3F710531F028F08EEF0E942F2422
:1051F0006FEF70E0688303C08DEF0E942F24DF9172
:10520000CF910895653671058105910518F00E94CA
:10521000C2230895209114023091150240E050E01D
:105220000E94B92F28EE33E040E050E00E94EC2FBE
:10523000CA01B9010E94392C0895DC0119968D919B
:105240009C911A97FC0125913491CD01F9010995A2
:105250000895DF92EF92FF920F931F93CF93DF9306
:10526000EC017A018B01DFB6F8942D853E858F85A0
:1052700098892817390711F080E001C08FEF8D8BD6
:10528000882381F02D853E858F85988928173907D9
:1052900021F0C90160E00E94B2248F8598896FEFE8
:1052A0000E94B22488858160888788858B7F888763
:1052B00088858D7F888789859A850496FC0125914C
:1052C0003491CE01B801A701F9010995DFBEDF9144
:1052D000CF911F910F91FF90EF90DF900895BF92B3
:1052E000CF92DF92EF92FF920F931F93CF93DF93B2
:1052F0007A018B01EC01BFB6F8944F3F8FEF58074E
:105300008FEF68078FEF780721F4A1E0CA2ED12C28
:1053100024C0CB01BA01F3E0660F771F881F991FE5
:10532000FA95D1F7209110023091110240911202AA
:1053300050911302620F731F841F951FA8019701DC
:10534000E4E0220F331F441F551FEA95D1F70E9456
:10535000EC2F69010894C108D10898A99923C9F1D3
:10536000ECA1FDA180819095892380838FEFE816C1
:105370008FEFF8068FEF08078FEF180719F421E079
:1053800030E01DC032E0EE0CFF1C001F111F3A95EB
:10539000D1F76091100270911102809112029091E8
:1053A00013026E0D7F1D801F911FEE0CFF1C001F4E
:1053B000111FA80197010E94EC2F215030402C159D
:1053C0003D0538F0ECA1FDA1808198A9892B80834F
:1053D0006901E8A5F9A5C082EAA5FBA5D082BFBEF8
:1053E000DF91CF911F910F91FF90EF90DF90CF90C1
:1053F000BF900895DC019696ED91FC91979780817E
:1054000087728083D0969C91D097992341F094968F
:10541000ED91FC91959780819095892380830895E3
:10542000DC0155968C915597882371F09696ED91F5
:10543000FC9197978081877B80839696ED91FC9174
:1054400097978081806980830895DC019C96ED9117
:10545000FC919D9760830895DC0155968C9155973A
:10546000882371F09696ED91FC91979780818F76C5
:1054700080839696ED91FC919797808188648083D4
:105480000895CF93DF93EC010E941D298D89882315
:1054900011F020E90CC08D859E85892B11F020E943
:1054A00001C020E08F859889892B09F02864EEA13E
:1054B000FFA12083DF91CF910895DC01262F149660
:1054C0008D919C911597892B59F01496ED91FC9133
:1054D000159716966D917C911797822F09950895CF
:1054E0009096ED91FC919197CD0109950895FC015D
:1054F00022A133A1F90109950895DF93CF930F926B
:10550000CDB7DEB7FC0180819181BE016F5F7F4F17
:105510000E946F2B882319F42FEF3FEF03C089817E
:10552000282F30E0C9010F90CF91DF910895CF93DC
:10553000DF93EC01888199810E94B72B882331F495
:1055400088858460888785EF0E942F24DF91CF9122
:105550000895DC0119968D919C911A970296FC0191
:1055600025913491CD01F90109950895CF93DF93E9
:10557000EC0188858E7F8887EE89FF89309721F03E
:10558000888D998D6FEF0995E985FA853896259173
:1055900034912115310519F0CE01F9010995DF91FA
:1055A000CF910895CF93DF93EC0188858160888740
:1055B000E985FA853A96259134912115310519F03E
:1055C000CE01F9010995EE89FF89309721F0888D88
:1055D000998D60E00995DF91CF910895EF92FF9248
:1055E0000F931F93CF93DF938C017B01EA010BC0D4
:1055F000D7016D917D01D8015C96ED91FC915D978D
:10560000C80109952197209799F7DF91CF911F91B4
:105610000F91FF90EF9008951F93FC01162F248D9A
:10562000358DF9010995812F1F910895FC01268D73
:10563000378DF90109950895FF920F931F93DF931A
:10564000CF930F92CDB7DEB78C01FFB6F894FC0173
:1056500082819381BE016F5F7F4F0E946F2B8823F1
:1056600029F0C80169810E94A92A07C0C8010E94C7
:10567000D22AF80180858D7F8087FFBE0F90CF9161
:10568000DF911F910F91FF9008950F931F93CF9378
:10569000DF93162FEC0102C00E94DD2B8A819B81D3
:1056A0000E94AF2B8823C1F70FB7F894888581FD3E
:1056B0000BC0888582608887CE010E94B62ACE0101
:1056C000612F0E94A92A05C08A819B81612F0E94B7
:1056D000B72B0FBFDF91CF911F910F910895CF93FB
:1056E000DF93DC01EB014FB7F894009799F1129624
:1056F0008D919C911397892B69F114968D919C91B2
:105700001597892B39F116962D913C911797ED91AC
:10571000FC911197E20FF31F808188832F5F3F4F29
:1057200017963C932E93169712968D919C911397F2
:105730002817390721F417961C921E921697149673
:105740008D919C911597019715969C938E93149724
:105750008FEF01C080E04FBFDF91CF9108950E948D
:105760006C2C892B11F080E008958FEF08951F9322
:10577000CF93DF93EC01462F1FB7F8942C813D8126
:105780006A817B812617370710F080E011C08E8177
:105790009F81820F931F0E94D82FE881F981E80F23
:1057A000F91F40838C819D8101969D838C838FEFAF
:1057B0001FBFDF91CF911F9108958FB7789400009C
:1057C0000000000000000000000000008FBF0895EE
:1057D000CF93DF939C010097E9F0FC0185919491B0
:1057E000FC01A591B4910296FC01C591D4912E5F64
:1057F0003F4FF90124918881822349F09FB7F894A3
:105800008C91209582238C939FBF000003C087EF6B
:105810000E942F24DF91CF910895CF93DF939C01B5
:105820000097E1F0FC0185919491FC01A591B49160
:105830000296FC01C591D4912E5F3F4FF90124914E
:105840008881822341F09FB7F8948C91822B8C93AE
:105850009FBF000003C087EF0E942F24DF91CF91EC
:105860000895662319F00E940D2C08950E94E82BDC
:105870000895613023E0720720E0820720E092075C
:1058800048F423E030E040E050E00E94EC2F2A95FD
:10589000F1F708959B01AC0182E056954795379545
:1058A00027958A95D1F7DA01C901203060E03607E3
:1058B00061E0460760E0560720F08FEF9FEFA0E021
:1058C000B0E0FC013197F1F7A0E0B0E0281B390B04
:1058D0004A0B5B0B41F70895FC014FB7F894009712
:1058E00019F420E030E006C0228133818481958163
:1058F000281B390B4FBFC90108956F927F928F9279
:105900009F92AF92BF92CF92DF92EF92FF920F934E
:105910001F93DF93CF93CDB7DEB72B970FB6F894D5
:10592000DEBF0FBECDBF5C014B017A01FC011782C7
:105930001682838181FD08C06FEF7FEF08C142E0CE
:1059400050E0E40EF51E04C03E010894611C711C79
:10595000F501D380F401D3FC8591D3FE81914F01F1
:10596000882309F4F1C0853259F4D3FC6591D3FE44
:1059700061914F01653219F0062F10E01BC085E2DE
:1059800090E02BC0002309F4DFC087E291E0602F94
:1059900070E00E94E12E892B39F4033211F410617A
:1059A00003C00C3661F41068F401D3FC0591D3FEFA
:1059B00001914F0117FFE6CF002309F4C5C080E233
:1059C00091E0602F70E00E94E12E892B51F044E0BD
:1059D00050E0E40EF51E8FE390E0B5010E941E2F0B
:1059E000B7CF033629F0033779F00335F1F40BC054
:1059F00087010E5F1F4FF70180819181B5010E94E1
:105A00001E2F7801A5CF1160F701C080D18004C09E
:105A100090E0B5010E941E2FF60110FD859110FF48
:105A200081916F018823A1F78ACF043611F00936DE
:105A300039F517FF08C0F701208131814281538178
:105A400084E090E00AC0F701808191819C014427A5
:105A500037FD4095542F82E090E0E80EF91E1F7E3E
:105A600057FF08C050954095309521953F4F4F4FB7
:105A70005F4F1064CA01B901A3012AE030E034C0CD
:105A80000037A9F0013730F40835B1F00F3609F0CE
:105A90005BC006C0053739F0083709F055C008C0AB
:105AA00028E030E00CC01F7E2AE030E008C0106122
:105AB000146220E130E003C0146020E132E017FFFF
:105AC00008C0F701608171818281938144E050E0D8
:105AD00008C0F70180819181BC0180E090E042E044
:105AE00050E0E40EF51EA3010E945B2FD82ED618BD
:105AF000012F10E006FF05C08DE290E0B5010E9485
:105B00001E2F04FF15C0FE01ED0DF11D80818033B5
:105B100079F080E390E0B5010E941E2F02FF08C0DB
:105B200000721070C801885A9F4FB5010E941E2F45
:105B3000DA94F301ED0DF11D808190E0B5010E9432
:105B40001E2FDD20A9F704CFF50166817781CB01F7
:105B50002B960FB6F894DEBF0FBECDBFCF91DF916D
:105B60001F910F91FF90EF90DF90CF90BF90AF907B
:105B70009F908F907F906F9008950F931F93CF9376
:105B8000DF93689F8001699F100D789F100D11248D
:105B9000C8010E94D92DEC01009729F060E070E067
:105BA000A8010E94F92ECE01DF91CF911F910F9194
:105BB0000895CF93DF93BC018230910510F462E029
:105BC00070E0A091E504B091E604ED01E0E0F0E0C2
:105BD00040E050E021C0888199818617970769F4D9
:105BE0008A819B81309719F09383828304C09093BC
:105BF000E6048093E504FE0134C06817790738F4A1
:105C00004115510519F08417950708F4AC01FE0100
:105C10008A819B819C01E9012097E9F64115510594
:105C2000A9F1CA01861B970B049708F4BA01E0E0BA
:105C3000F0E02AC08D919C91119784179507F9F493
:105C40006417750781F412968D919C911397309784
:105C500019F09383828304C09093E6048093E50453
:105C6000FD0132964FC0CA01861B970BFD01E80F5C
:105C7000F91F6193719302978D939C9343C0FD012B
:105C8000828193819C01D9011097A1F68091E30450
:105C90009091E404892B41F48091E3029091E40215
:105CA0009093E4048093E3044091E5025091E6026E
:105CB0004115510541F44DB75EB78091E1029091D5
:105CC000E202481B590B2091E3043091E4042417AD
:105CD0003507B0F4CA01821B930B8617970780F033
:105CE000AB014E5F5F4F8417950750F0420F531F73
:105CF0005093E4044093E304F9016193719302C06B
:105D0000E0E0F0E0CF01DF91CF910895CF93DF93F2
:105D1000009709F450C0EC0122971B821A82A091CF
:105D2000E504B091E604109709F140E050E0AC17AB
:105D3000BD0708F1BB83AA83FE0121913191E20FD7
:105D4000F31FAE17BF0779F48D919C911197280F1F
:105D5000391F2E5F3F4F3983288312968D919C9176
:105D600013979B838A834115510571F4D093E60400
:105D7000C093E50420C012968D919C911397AD01BC
:105D8000009711F0DC01D3CFFA01D383C2832191B4
:105D90003191E20FF31FCE17DF0769F488819981F3
:105DA000280F391F2E5F3F4FFA01318320838A81EC
:105DB0009B8193838283DF91CF910895F8940C9413
:105DC0002F30FC010590061621F00020D9F7C00104
:105DD00008953197CF010895FB01DC0104C08D9136
:105DE0000190801921F441505040C8F7881B990B4D
:105DF0000895DC0101C06D9341505040E0F70895D3
:105E00000F931F93DF93CF93CDB7DEB70F81188524
:105E10009E01255F3F4FF801838188608383C8011D
:105E200069857A85A9010E947D2CF8012381277F4D
:105E30002383CF91DF911F910F9108950F931F93AB
:105E4000CF93DF938C01EB018B8181FF1BC082FF1D
:105E50000DC02E813F818C819D812817390764F404
:105E6000E881F9810193F983E88306C0E885F98523
:105E7000802F0995892B31F48E819F8101969F8314
:105E80008E8302C00FEF1FEFC801DF91CF911F91EA
:105E90000F9108950F931F938C01FC0183818860FB
:105EA0008383C8010E947D2CF8012381277F2383EF
:105EB0001F910F910895FA01AA27283051F120313E
:105EC00081F1E8946F936E7F6E5F7F4F8F4F9F4F8E
:105ED000AF4FB1E03ED0B4E03CD0670F781F891FD0
:105EE0009A1FA11D680F791F8A1F911DA11D6A0F9E
:105EF000711D811D911DA11D20D009F468943F9151
:105F00002AE0269F11243019305D3193DEF6CF014F
:105F10000895462F4770405D4193B3E00FD0C9F715
:105F2000F6CF462F4F70405D4A3318F0495D31FD82
:105F30004052419302D0A9F7EACFB4E0A6959795D5
:105F4000879577956795BA95C9F7009761057105AB
:105F500008959B01AC010A2E0694579547953795F5
:105F60002795BA95C9F7620F731F841F951FA01D4F
:105F70000895629FD001739FF001829FE00DF11D93
:105F8000649FE00DF11D929FF00D839FF00D749FB3
:105F9000F00D659FF00D9927729FB00DE11DF91F5F
:105FA000639FB00DE11DF91FBD01CF0111240895BC
:105FB000AA1BBB1B51E107C0AA1FBB1FA617B7072F
:105FC00010F0A61BB70B881F991F5A95A9F780954B
:105FD0009095BC01CD010895A1E21A2EAA1BBB1B0E
:105FE000FD010DC0AA1FBB1FEE1FFF1FA217B307A5
:105FF000E407F50720F0A21BB30BE40BF50B661FBB
:10600000771F881F991F1A9469F76095709580957E
:1060100090959B01AC01BD01CF01089597FB092E1E
:1060200005260ED057FD04D0D7DF0AD0001C38F467
:1060300050954095309521953F4F4F4F5F4F0895B4
:10604000F6F790958095709561957F4F8F4F9F4F94
:106050000895EE0FFF1F0590F491E02D0994F89438
:02606000FFCF70
:106062000A1168656C6C6F20776F726C6421000690
:106072000024F400803E1000B902C50200000000B6
:10608200003407FFFFB706BA06BD0DC20D000000BF
:1060920000000000452B1C2B972A7D2AC000C1005E
:1060A200C400C500C60000000208CC0600BD06C937
:1060B2000600000000D20600FF00000000000022DF
:1060C20007A4060100020000000000CF06000080C5
:1060D200000000AB06DC05F4010000000000000037
:1060E200000000A606010000000000000000000001
:1060F20000000200000000D10C00000000000000BF
:106102000200000000D10C000000000000000100AD
:106112000000000000DE0C000077035000000000C9
:106122000000000000C70350000000000000000053
:10613200008A250000000200000000CC25AF2500E7
:08614200002000EE0400000043
:00000001FF
